:03000000023B843C
:0C3B840078FFE4F6D8FD758155023BCBBC
:102377000A53746172743A20004950436F6E6E6558
:1023870063745245510A00444843502D4F4B0A008D
:102397004950436F6E6E65637400C0E4E0EFF2E589
:1023A700F020D1E8EDEAEEEC4950285243290A0023
:1023B700C2E5F0F1E8FF20495020ECEEE4F3EBFF33
:1023C7003A20322E3420EEF22032302E31312E32A6
:1023D7003030350A00C4E0F2E020F1EEE7E4E0ED4A
:1023E700E8FF3A200053657020323620323030360D
:1023F70000200031313A32313A3437000A000A50AE
:10240700524F473A20202020202020202020202023
:1024170020202020202020202020202020202020B5
:1024270020202020202020202020202020202020A5
:102437002020202020202020202020202020202095
:102447002020202020202020200A0044756D70586D
:1024570020202020203030203031203032203033EF
:1024670020303420303520303620303720303820A7
:102477003039203041203042203043203044203052
:10248700452030460A003A200044756D70442020EC
:10249700202020303020303120303220303320309F
:1024A700342030352030362030372030382030394E
:1024B7002030412030422030432030442030452016
:1024C70030460A00457272206B65790052642065B8
:1024D7006570726F6D0A005264204D454D0A0044C5
:1024E700656275674950204F4E0A004465627567FB
:1024F7004950204F46460A00446562756755736523
:1025070072204F6E0A0044656275675573657220C5
:102517004F46460A0044656275674D7367204F6EE4
:102527000A0044656275674D7367204F46460A0087
:10253700436F6E666967206C6F636B210A00577281
:1025470020656570726F6D0A00205361766520659E
:102557006570726F6D210A00457272204D414321EB
:10256700004C6F61643E3E00576169745265737435
:1025770061727421004E4F4950004C494E4B434FF6
:102587004E5452005452415353004652004E4F4C42
:10259700494E4B00494E490000FF257CFF2581FF2E
:0E25A700258BFF2591FF2594FF259BFF259F87
:06443B00015200015000D7
:10438D00C2AFC28E758900438910758BFF758DB7CD
:07439D00D2ABD28ED2AF2299
:03001B00023A5F47
:103A5F00C0E0C083C082C0D0C2AFC28E758BFF756D
:103A6F008DB720190675A61E75A6E10550D215E56E
:103A7F0052600205520555E555540F7053D220E59B
:103A8F0055543F7014D213906E48E0600C04F0E070
:103A9F00D394B44004C2AF80FE906E43E060020442
:103AAF00F0E551D3940140021551906940E0600256
:103ABF0014F0906E49E0D394014003E014F03018F5
:103ACF00020553E554D394644004D219800205547F
:103ADF00E54FD394014002154FD28ED2AFD0D0D044
:063AEF0082D083D0E0321A
:10413C00E4FFFEFD74162DF582E4346BF583E02F5D
:10414C00FFE43EFE0DBD10ECE4FD746B2DF582E436
:10415C003469F583E0FC2FFFE43EFEEC60040DBDFA
:02416C0080E8E9
:01416E00222E
:100A1A00C21D7D027C007F071243548F3CE53C6473
:100A2A006060097D017F601242A7D21DE4FDFC7F50
:100A3A000B1243548F3CE53C30E6097D04E4FF1277
:100A4A0042CBD21D7D017C007F071243548F3CE5C7
:100A5A003C7008FD7FFF1242A7D21D301D031260B1
:100A6A0000C2AFC288D2A8C2AA123AF5D2AF1241C6
:100A7A003C1227C61230EDC219123FC2906B14E025
:100A8A00C3940350037403F0D21FD21ED21DD29313
:100A9A00201D077E237F771231E0E4906D34F01237
:100AAA00438DC2AF755101A3F0C21AC21BD2AF75F2
:100ABA00A70775A61E75A6E1124371201D19AF3C42
:100ACA007E007D031232C5E4FF1238787E6B7F34D4
:100ADA00E4FB7D01123481906E48E060037401F0FA
:100AEA00E4906940F0A37455F0A37481F0E4F553DF
:100AFA00E4F554906940E070031225B5906E49E020
:100B0A00B401119080007410F0E4906E49F0D21D87
:100B1A00D21ED21FE553D39403402D908002E4F0F5
:100B2A00908001F0908000F0E553D394054003745F
:100B3A0001F0E553D3940A400FE4F553C216906DC1
:100B4A0035F0755101123FC29080A0E070077FCB4B
:100B5A007E03123D9F9080B8E07003123926908080
:100B6A00D0E07014302111906E3F74FFF0906B0842
:100B7A00E0FEA3E0FF123E9F908000E07013301A5F
:100B8A0010122FE1906AF0EFF0D394004003121193
:100B9A0010908002E07006908000E06005D2180292
:100BAA000AFAC218E4F553906940E06003020AFAAF
:100BBA00301C15122E7A906AF0EFF0D39400400898
:100BCA00301405E0FF1243F2201B03020DD9122C48
:100BDA00FD906AF0EFF07003020AFA906E48E06046
:100BEA00037401F0906B34E054BF247F7003020C4D
:100BFA00AD147003020C8E24026003020D84201DC2
:100C0A00077E237F801231E0906B0CE0FF70069024
:100C1A006B10E06055906E3FE0FEB50722A3E0FF3F
:100C2A00906B0DE0B50718906E41E0FF906B0EE0F7
:100C3A00B5070C906E42E0FF906B0FE06F602B904F
:100C4A006B10E06E7035906E40E0FF906B11E0B56E
:100C5A000729906E41E0FF906B12E0B5071D906E78
:100C6A0042E0FF906B13E0B50711C216906D357420
:100C7A0003F0120021755101020DD9906E3F74FFE5
:100C8A00F0020DD9906E37E0FF906B36E06F60038B
:100C9A00020DD9906E37E004F0E4F551906D34F00E
:100CAA00020DD9301603020DD9906B35E0D3940AA0
:100CBA005003020D57A3E064026003020D57906AC5
:100CCA00FDE0FF906B3FE06F6003020AFA906AFE54
:100CDA00E0FF906B40E06F6003020AFA906AFFE05F
:100CEA00FF906B41E06F6003020AFA906B00E0FF2D
:100CFA00906B42E06F6003020AFA906B01E0FF908A
:100D0A006B43E06F6003020AFA906B02E0FF906B9C
:100D1A0044E06F6003020AFA7E237F8E1231E0906C
:100D2A006B3763A201906AF563A2017F12122A82CD
:100D3A00906B4963A201906E3F63A2017F04122A5D
:100D4A0082906D357406F0755102020AFA740344F2
:100D5A006B7003020AFA124450D216E4F551906DF0
:100D6A0034F0906E4304F0E4906E36F0A3F0201D48
:100D7A005E7E237F971231E08055301652906B3495
:100D8A00E020E74B906B36E0FF906E36E0FE6F6036
:100D9A000D906E3EE07007EE146F70338013906E04
:100DAA0036E004F0906AF0E0FFD394044003124165
:100DBA000890683C7482F0A37401F0906B36E0905E
:100DCA00683EF07E687F3C7D03123E20020AFA20CC
:100DDA001603020E959080D0E0700B906B08E0FE2F
:100DEA00A3E0FF123E9FE5517066906E43E0D394F4
:100DFA003C4037906E3EE07031120006906E4374AC
:100E0A0001F0E4906C34F0A37412F0906E37E09025
:100E1A006C36F0A374FDF090694363A201906C38BC
:100E2A0063A2017F12122A82800612416FEF6020AC
:100E3A007E6C7F34906C35E02404FD123E20906E67
:100E4A003EE06003020AFA906B14E0F551020AFAD6
:100E5A00124428EF601590683C7483F0E4A3F07E96
:100E6A00687F3C7D02123E20020AFAE55164016065
:100E7A0003020AFA906D34E004F0E0C3940540B02E
:100E8A00C216E4A3F0120021020AFAE551640160D5
:100E9A0003020AFA906D35E0147003020F391470D8
:100EAA0003020F6514700302100D1470030210C3BD
:100EBA0024FE606924066003020AFAE4F553F53C4D
:100ECA0074EC253CF582E43469F583E0FF74F5257A
:100EDA003CF582E4346AF583EFF0053CE53CB43F27
:100EEA00DF202121906B0C63A201906E3F63A20167
:100EFA007F04122A82906D357401F0906D34F0757A
:100F0A005103020AFA906D357404F0906D3474013D
:100F1A00F0755114906E3F74FFF0020AFAE4F5532B
:100F2A00123FC2906D357401F0755103020AFA90AE
:100F3A006E3FE0600B906B08E0FEA3E0FF123E9F5D
:100F4A00755102906D357402F0906B03E0700302E4
:100F5A000AFA906D357403F0020AFA906E3FE07057
:100F6A0003020FFE906C347480F0906C367402F0B9
:100F7A00E4A3F0A304F0906AFD63A201906C3963C4
:100F8A00A2017F0A122A82906C437430F0A3747B08
:100F9A00F0E4F53C746B253CF582E43469F583E0B2
:100FAA00FF60117445253CF582E4346CF583EFF05B
:100FBA00053C80E07445253CF582E4346CF5837485
:100FCA007DF07446253CF582E4346CF583E4F0E563
:100FDA003C2411906C35F07C6E7D3F906B08E0FAF2
:100FEA00A3E0FB7F02123D1B7E6C7F34E53C241399
:100FFA00FD123E20906D357404F0906B14E0F551AB
:10100A00020AFA906E3FE070030210B4906C3474D6
:10101A0080F0906C367401F0E4A3F0A304F0A3749A
:10102A0030F0A3747BF0E4F53C746B253CF582E464
:10103A003469F583E0FF6011743B253CF582E434A2
:10104A006CF583EFF0053C80E0743B253CF582E4C7
:10105A00346CF583747DF0743C253CF582E4346C81
:10106A00F583E4F0E53C2407906C35F07C6E7D3F17
:10107A00906B08E0FAA3E0FB7F02123D1B7E6C7FB7
:10108A0034E53C2409FD123E20906E3EE0601B12BE
:10109A004450D216E4F551906D34F0906E4304F04A
:1010AA00E4906E36F0A3F0020AFA906D357404F0FB
:1010BA00906B14E0F551020AFA906E3FE0FF600966
:1010CA00F460069080027410F020212B7551029072
:1010DA006D34E06401FFF0A37401F0EF6005906BDA
:1010EA000C8003906B1063A201906E3F63A2017F94
:1010FA0004122A82020AFA755114906E3F74FFF0A4
:05110A00020AFA80FE5C
:01110F0022BD
:10111000906B35E0B444047F0180027F00906B3413
:10112000E0B447047E0180027E00EE5F604A906A70
:10113000FDE0906B36F0906AFEE0906B37F0906ABD
:10114000FFE0906B38F0906B00E0906B39F0906BA3
:1011500001E0906B3AF0906B02E0906B3BF0906B8B
:10116000357452F0906AEA63A2019080A863A201EC
:101170007F06122A8202161E906AF0E0C39408507D
:1011800003021627906AFDE0FF906B36E06F600364
:10119000021627906AFEE0FF906B37E06F60030253
:1011A0001627906AFFE0FF906B38E06F600302162D
:1011B00027906B00E0FF906B39E06F600302162709
:1011C000906B01E0FF906B3AE06F6003021627908E
:1011D0006B02E0FF906B3BE06F6003021627906E9E
:1011E00048E060037401F0906E497464F0906B35D0
:1011F0007452F0906B34E0644D703C7E237FA112FA
:1012000031E07E237FB71231E01244337E237FDC4E
:101210001231E07E237FEC1231E07E237FF8123121
:10122000E07E237FFA1231E07E247F031231E07EDC
:10123000247F051231E022906B34E0644C70527EC2
:10124000247F521231E0906B3CE0F53DA3E0F53E87
:10125000E4F53F7D03AF3EAE3D1232C57E247F8D67
:101260001231E0AE3DAF3EE4FB7D101234817E24AE
:101270007F031231E07410253EF53EE4353DF53D27
:10128000053FE53FC3941040CA7E247F031231E03E
:1012900022906B34E0646C705CF5417E247F901288
:1012A00031E0E4F540AF417E007D031232C57E247B
:1012B0007F8D1231E0E4F53FA841E6FF743E253F03
:1012C000F582E4346BF583EFF00541053FE53FB46B
:1012D00010E67E6B7F3EE4FB7D101234817E247F1E
:1012E000031231E00540E540C3940840B87E247FF6
:1012F000031231E022906B34E0644B7046F53F748A
:1013000026253FF582E4346BF583E0FF6016743CDC
:10131000253FF582E4346BF583E0B50710053FE522
:101320003FB408DB9069407432F002161E906B34B3
:101330007421F0301D0302161E7E247FCB1231E093
:1013400002161E906B34E06452704E201D077E24FE
:101350007FD31231E0906B3DE0906AF0F0E4F53F0E
:10136000906AF0E0FDE53FC39D5022906B3CE02584
:101370003F24EBF582E43469F583E0FF743E253FBA
:10138000F582E4346BF583EFF0053F80D37E6B7F0D
:1013900034ED240AFD123C1022906B34E064497055
:1013A00045201D077E247FDE1231E0906B3CE0F586
:1013B0003DA3E0F53EE4F53F853E82853D83E0FFB9
:1013C000743E253FF582E4346BF583EFF0053EE58E
:1013D0003E7002053D053FE53FB480DC7E6B7F3407
:1013E0007D8A123C1022906B34E064446003021446
:1013F00077906B3CE0FF6444700302161EEFB4313B
:101400000CC21D7E247FE61231E002161E906B3C5A
:10141000E0B4300CD21D7E247FF21231E002161EA1
:10142000906B3CE0B4320CD21E7E247FFF1231E080
:1014300002161E906B3CE0B4330CC21E7E257F0D5D
:101440001231E002161E906B3CE0B4340CD21F7EC9
:10145000257F1C1231E002161E906B3CE0B4350C67
:10146000C21F7E257F291231E002161E906B3CE0E0
:10147000FF12001E02161E906940E07013201D0727
:101480007E257F371231E0906B347421F002161EF6
:101490009069407432F0906B34E0FFB45104C2AFF5
:1014A00080FEEF64577045201D077E257F45123171
:1014B000E0906B3DE0906AF0F0E4F53F906AF0E078
:1014C000FFE53FC39F400302161E743E253FF58291
:1014D000E4346BF583E0FF906B3CE0253F24EBF5B3
:1014E00082E43469F583EFF0053F80D0906B34E0FF
:1014F00064536003021599201D077E257F50123129
:10150000E0906AFDE0FF9069F4E06F703C906AFE45
:10151000E0FF9069F5E06F7030906AFFE0FF90693E
:10152000F6E0B50724906B00E0FF9069F7E0B5079F
:1015300018906B01E0FF9069F8E0B5070C906B0222
:10154000E0FF9069F9E06F6016906B347421F03021
:101550001D0302161E7E257F5F1231E002161EE477
:10156000F53FE4F55474EB253FF582E43469F583E7
:10157000E0FDAF3F124200053FE53FC394FE40E26D
:10158000C2AFE4907FF0F0A3F0907FFD74AAF0A3C7
:1015900074FFF0A37455F080FE906B34E0644F70DC
:1015A0004B906B3CE0F53DA3E0F53EE53E453D70DC
:1015B0000A201D077E257F681231E0201D077F2A43
:1015C0007E001231E0E4F53F743E253FF582E434BD
:1015D0006BF583E0853E82853D83F0053EE53E70F8
:1015E00002053D053FE53FB480DE8032906B34E07C
:1015F000B4452B201D077E257F6F1231E0906B3C98
:10160000E0FFA3E0907FF0CFF0A3EFF0C2AF907FB8
:10161000FD74AAF0A374FFF0A37455F080FE7E6BF6
:071620007F347D08123C102D
:0116270022A0
:1040D000AE07EEC39430400BEED394395005EE2476
:1040E000D0FF22EEC39461400BEED394665005EEF0
:1040F00024A9FF22EEC39441400BEED39446500511
:08410000EE24C9FF22AF0622E4
:1027C600C214E4906E48F0D221C217906E3EF0908B
:1027D6006AFD63A201906E3863A2017F06122A8207
:1027E600E4F53DE53D75F003A424A0F582E4342527
:1027F600F583E493FB740193FA740293F91220E3D0
:1028060070030229A6E4F53EF53FFD746B2DF582B3
:10281600E43469F583E0FF70030229A1E53D75F014
:1028260003A424A0F582E43425F583E493FB740124
:1028360093FA740293F9853E827583001220FCFE9A
:10284600EFB50608753F01053E02299DE53F700379
:1028560002299DEE6003022998E53D24FE602214BC
:10286600700302298814700302298C14700302294C
:1028760094240460030229A1906E487401F0022991
:10288600A1D214746B2DF582E43469F583E0FF64FC
:102896002D70030229A11240D0EFC454F0FC746CD1
:1028A6002DF582E43469F583E0FF1240D0EF2C90D9
:1028B6006E38F0746D2DF582E43469F583E0FF120D
:1028C60040D0EFC454F0FC746E2DF582E43469F503
:1028D60083E0FF1240D0EF2C906E39F0746F2DF527
:1028E60082E43469F583E0FF1240D0EFC454F0FC73
:1028F60074702DF582E43469F583E0FF1240D0EF61
:102906002C906E3AF074712DF582E43469F583E00B
:10291600FF1240D0EFC454F0FC74722DF582E434FB
:1029260069F583E0FF1240D0EF2C906E3BF0747394
:102936002DF582E43469F583E0FF1240D0EFC454EC
:10294600F0FC74742DF582E43469F583E0FF1240DF
:10295600D0EF2C906E3CF074752DF582E43469F559
:1029660083E0FF1240D0EFC454F0FC74762DF5825C
:10297600E43469F583E0FF1240D0EF2C906E3DF011
:102986008019D2178015906E3E7401F0800DC22119
:102996008009E4F53FF53E0D022811053D0227E9C1
:0129A600220E
:03000300023F06B3
:0D3F0600C0E0C083C082C0D075D000C007ED
:103F1300C2A8908008E0FFEF54F06035EF30E4086A
:103F2300D21A9080087410F0EF30E508D21C90800C
:103F3300087420F0EF30E608D21B9080087440F03C
:103F4300EF30E7069080087480F0908008E0FF80EF
:093F5300C690800874FFF0D2A8AA
:0B3F5C00D007D0D0D082D083D0E0325C
:103FC2009080007480F0906AF563A201F583F58217
:103FD20063A2017F08122A82906AFD63A201908087
:103FE2008863A2017F0A122A82906B07E0FF908009
:103FF200B1F09080E1EFF09080957455F0A3F090CD
:0C40020080007401F09080097470F022BE
:043D9F00AD07AC06BA
:103DA300908009E04410F09080A0E0706F9080A1B3
:103DB3007482F09080A874FFF0A3F0A3F0A3F0AF97
:103DC30004AE079080AEEEF0AE05A3EEF0AE079022
:103DD30080ACEEF0AE05A3EEF09080007402F0909C
:103DE3006F6812228D00000000906F68E0908040A1
:103DF300F0906F69E0908041F0906F6AE0908042AC
:103E0300F0906F6BE0908043F0A3E4F0A3F0A3F095
:0C3E1300A3F0908018F0A3F0A3F0A3F03F
:013E1F002280
:043E9F00AD07AC06B9
:103EA300908009E04440F09080D0E070559080D13C
:103EB3007482F0AF049080DEEFF0AF05A3EFF090D3
:103EC30080027402F0906F6C12228D00000000904B
:103ED3006F6CE0908058F0906F6DE0908059F09097
:103EE3006F6EE090805AF0906F6FE090805BF0A36C
:103EF300E4F0A3F0A3F0A3F0908030F0A3F0A3F0DC
:023F0300A3F029
:013F05002299
:10392600908009E04420F09080B8E060030239C737
:103936009080B97482F07F039080C6EFF07FCDA3AC
:10394600EFF07F039080C4EFF0A374CDF030022235
:10395600906B0CE09080C0F0906B0DE09080C1F011
:10396600906B0EE09080C2F0906B0FE09080C3F0F9
:10397600800C9080C074FFF0A3F0A3F0A3F09080B9
:10398600017402F0906F7012228D00000000906F9B
:103996006CE090804CF0906F6DE090804DF0906FF1
:1039A6006EE090804EF0906F6FE090804FF0A3E451
:1039B600F0A3F0A3F0A3F0908024F0A3F0A3F0A36B
:0139C600F010
:0139C70022DD
:103D1B008C3D8D3EA907EAFDE975F018A424ACFF94
:103D2B00E5F034808F82F583EDF0EBFDE975F0184B
:103D3B00A4FFAEF024ACFBEE34808B82F583A3EDB5
:103D4B00F0853E828C83E0FDEF24A8FFEE3480FEED
:103D5B008F82F583EDF0853E828C83A3E08F828E7C
:103D6B0083A3F0853E82853D83A3A3E0FDE975F037
:103D7B0018A424A8FFE5F03480FE8F82F583A3A35B
:103D8B00EDF0853E828C83A3A3A3E08F828E83A369
:043D9B00A3A3F022CC
:063C10008D42AB07AA067D
:103C1600906F68E0FCA3E0FDA3E0FEA3E0F5468E0E
:103C2600458D448C43AE02AF038E838F8263A2011F
:103C3600E545540744C0F58385468263A201AF4239
:103C4600122AEB908000E020E5F9E4FCFDFEE54653
:103C56002542F546EE3545F545ED3544F544EC355A
:103C660043F543C2A8908040E543F0A3E544F0A3A2
:103C7600E545F0A3E546F0D2A89080007420F0AFA9
:0F3C860046AE45AD44AC43906F68122281AF4209
:013C9500220C
:063E20008D3DAB07AA0670
:103E2600906F6CE0FCA3E0FDA3E0FEA3E0F5418EFD
:103E3600408D3F8C3EAE02AF038E838F8263A2011C
:103E4600E540540744D0F58385418263A201AF3D26
:103E5600122AEBE4FCFDFEE541253DF541EE354039
:103E6600F540ED353FF53FEC353EF53EC2A8908076
:103E760058E53EF0A3E53FF0A3E540F0A3E541F0A9
:103E8600D2A89080027420F0AF41AE40AD3FAC3E68
:083E9600906F6C122281AF3D18
:013E9E002201
:023878008F3E81
:10387A00908001E030E5037F0022906F70E0FCA3A6
:10388A00E0FDA3E0FEA3E0F5428E418D408C3F901F
:10389A006E3863A201E541540744C8F58385428224
:1038AA0063A2017F06122B01E5422406F542E435A4
:1038BA0041F541E43540F540E4353FF53F906D363A
:1038CA0063A201E541540744C8F58385428263A295
:1038DA0001AF3E122B01E4FCFDFEE542253EF54216
:1038EA00EE3541F541ED3540F540EC353FF53FC247
:1038FA00A890804CE53FF0A3E540F0A3E541F0A392
:10390A00E542F0D2A89080017420F0AF42AE41ADFA
:0B391A0040AC3F906F70122281AF3E66
:01392500227F
:102FE100C2A89081E0E0F53D053D053D053D053D6B
:102FF100053D053D053D053D053D053D908010E044
:10300100F540A3E0F541A3E0F542A3E0F54390814B
:10301100E1E0F53D053D053D053D053D053D053D30
:10302100053D053D053D053D908014E0F544A3E0D7
:10303100F545A3E0F546A3E0F547D2A8E546B5423C
:1030410008E547B543037F0022E4F53DE546540713
:1030510044E0F58385478263A201906B3463A2014A
:103061007F08122B19906B3663A201906AEA63A262
:10307100017F06122A82906B34E0F53EA3E0F53F12
:10308100E4F53D906B34E0702AA3E024F8F53DE5CA
:1030910046540744E0F58385478274082582F5820A
:1030A100E43583F58363A201906B3463A201AF3DE4
:1030B100122B19AE3EE4FCFDE547253FF547E546F9
:1030C1003EF546ED3545F545EC3544F544C2A8904D
:1030D1008014E544F0A3E545F0A3E546F0A3E547F8
:0B30E100F0D2A89080007440F0AF3DDA
:0130EC0022C1
:102CFD00C2A89081E6E0F53D053D053D053D053D4C
:102D0D00053D053D053D053D053D053D908028E012
:102D1D00F540A3E0F541A3E0F542A3E0F543908132
:102D2D00E7E0F53D053D053D053D053D053D053D11
:102D3D00053D053D053D053D90802CE0F544A3E0A6
:102D4D00F545A3E0F546A3E0F547D2A8E4F53DE54A
:102D5D0046B5420AE547B54305C21B022E5BE54663
:102D6D00540744F0F58385478263A201906B346369
:102D7D00A2017F08122B19906B34E0F53EA3E0F50C
:102D8D003FE53F453E70099080027410F07F0022B0
:102D9D00906E3FE0FFF4602D906B36E06F70769093
:102DAD006E40E0FF906B37E06F706A906E41E0FF10
:102DBD00906B38E06F705E906E42E0FF906B39E083
:102DCD006F60228050906B36E0906E3FF0906B37C5
:102DDD00E0906E40F0906B38E0906E41F0906B3962
:102DED00E0906E42F0906B34E0702AA3E024F8F589
:102DFD003DE546540744F0F58385478274082582E6
:102E0D00F582E43583F58363A201906B3463A201EF
:102E1D00AF3D122B19AE3EE4FCFDE547253FF547CE
:102E2D00E5463EF546ED3545F545EC3544F544AF03
:102E3D0043AE42AD41AC40AB47AA46A945A844D3E9
:102E4D0012227040099080027410F07F0022C2A8F7
:102E5D0090802CE544F0A3E545F0A3E546F0A3E50D
:0C2E6D0047F0D2A89080027440F0AF3D06
:012E79002236
:102E7A00C2A89081E3E0F53D053D053D053D053DD0
:102E8A00053D053D053D053D053D053D90801CE0A0
:102E9A00F540A3E0F541A3E0F542A3E0F5439081B4
:102EAA00E4E0F53D053D053D053D053D053D053D96
:102EBA00053D053D053D053D908020E0F544A3E034
:102ECA00F545A3E0F546A3E0F547D2A8E4F53DE5CC
:102EDA0046B5420AE547B54305C21C022FC2E5467C
:102EEA00540744E8F58385478263A20190684063EA
:102EFA00A2017F0E122B2F906840E0F53EA3E0F569
:102F0A003F906E38E0FF906848E06F706C906E39C1
:102F1A00E0FF906849E06F7060906E3AE0FF906859
:102F2A004AE06F7054906E3BE0FF90684BE06F7020
:102F3A0048906E3CE0FF90684CE06F703C906E3DAC
:102F4A00E0FF90684DE06F7030906840E0702AA30F
:102F5A00E024F2F53DE546540744E8F583854782C7
:102F6A00740E2582F582E43583F58363A2019068A5
:102F7A004063A201AF3D122B2FAE3EE4FCFDE547B4
:102F8A00253FF547E5463EF546ED3545F545EC3531
:102F9A0044F544AF43AE42AD41AC40AB47AA46A963
:102FAA0045A844D31222705006E53F453E70099069
:102FBA0080017410F07F0022C2A8908020E544F0BE
:102FCA00A3E545F0A3E546F0A3E547F0D2A8908033
:062FDA00017440F0AF3D60
:012FE00022CE
:0431E0008E438F4447
:1031E400906F68E0FCA3E0FDA3E0FEA3E0F54A8E47
:1031F400498D488C47E54AFFE5495407FEE42FF51D
:1032040046EE34C0F545854682F5837423F00546C1
:10321400E546700205455345C7F582854583740A22
:10322400F00546E546700205455345C7906AFD63BF
:10323400A20185458385468263A2017F06122AEB9B
:1032440074062546F546E43545F5458543838544AE
:103254008263A20185458385468263A201122ACF37
:10326400908000E020E5F9E4FCFDFE906F68E0F852
:10327400A3E0F9A3E0FAA3E02FFFEE3AFEED39FD57
:10328400EC38FCEF2408FFE43EFEE43DFDE43CFCA6
:10329400906F68122281C2A8906F68E0908040F01D
:1032A400906F69E0908041F0906F6AE0908042F006
:1032B400906F6BE0908043F0D2A89080007420F06F
:0132C40022E7
:063481008E438F448D45CF
:10348700906F68E0FCA3E0FDA3E0FEA3E0F54B8EA0
:103497004A8D498C48E54BFFE54A5407FEE42FF572
:1034A70047EE34C0F546854782F5837423F0054718
:1034B700E547700205465346C7F582854683EBF01C
:1034C7000547E547700205465346C7906AFD63A264
:1034D7000185468385478263A2017F06122AEB7422
:1034E700062547F547E43546F546854383854482F7
:1034F70063A20185468385478263A201AF45122AED
:10350700EB908000E020E5F974082545F545FFE4D8
:10351700FCFDFEE54B2FF54BEE354AF54AED3549F7
:10352700F549EC3548F548C2A8908040E548F0A336
:10353700E549F0A3E54AF0A3E54BF0D2A890800057
:103547007420F0AF4BAE4AAD49AC48906F68122279
:0135570081F2
:013558002250
:0632C5008E428F43AB05B1
:1032CB00906F68E0FCA3E0FDA3E0FEA3E0F5498E60
:1032DB00488D478C46E549FFE5485407FEE42FF53A
:1032EB0045EE34C0F544854582F5837423F00545DE
:1032FB00E545700205445344C7F582854483EBF0E2
:10330B000545E54570020544906AFD63A2018544BD
:10331B008385458263A2017F06122AEB740625453D
:10332B00F545E43544F5445344C7E542854582856C
:10333B004483F00545E545700205445344C7F582C7
:10334B00854483E543F00545E54570020544534448
:10335B00C7908000E020E5F9E549240AF549E435FA
:10336B0048F548E43547F547E43546F546C2A8909D
:10337B008040E546F0A3E547F0A3E548F0A3E54917
:10338B00F0D2A89080007420F0AF49AE48AD47ACA6
:07339B0046906F68122281C9
:0133A2002208
:103AF500E4F53DE53D04FF12422A74F5253DF582C6
:103B0500E4346AF583EFF0053DE53DC3943F40E3BA
:103B1500E4F53DE53D247FFF12422A746B253DF512
:103B250082E43469F583EFF0746B253DF582E43466
:103B350069F583E0701D746B253DF582E43469F504
:103B4500837420F0746C253DF582E43469F583E4D3
:103B5500F08009053DE53DC3948040B7E49069EAEE
:103B6500F0F53DAF3D12422A74EB253DF582E43474
:0E3B750069F583EFF0053DE53DC394FE40E5A4
:013B8300221F
:10433400E4FDFCC3ED9FEC9E5015E4FBFA0BBB00BF
:0F434400010ABA01F8BB90F50DBD00010C80E431
:014353002247
:0D4401004390014390025390FE5390FD2222
:0D440E005390FD5390FE4390024390012215
:0E43E3005390FD439002E5905408FF5390FD67
:0143F10022A9
:0D441B005390FD4390014390025390FD2209
:07444200AE071FEE70FA2225
:0241D400AD0735
:1041D600E4FC5390FDEDA804088002C333D8FC30FC
:1041E600E70543900180035390FE7F051244424346
:0941F60090020CBC08DC5390FDA2
:0141FF00229D
:10427E00E4FF5390FD7E07439002E59030E00D740D
:10428E0001A806088002C333D8FC42075390FD1ED6
:08429E00C3EE6480948050DF40
:0142A60022F5
:10420000AB05AA071244017FA01241D41243E3AFC9
:10421000021241D41243E3AF031241D41243E3121A
:0A422000440E7F0A7E001243342290
:02422A00AB07E0
:10422C001244017FA01241D41243E3AF031241D4D4
:10423C001243E31244017FA11241D41243E3124210
:07424C007E12441B12440E18
:014253002248
:10435400A2AF9227C2AF8C838D82EF122B4743A268
:0C43640020122B4953A2DFA22792AFFFCA
:01437000222A
:0242A7008F3D49
:1042A900A2AF9227C2AFE4F5838D827406122B4721
:1042B900E53D43A220122B4953A2DFA22792AF7FEB
:0142C90001F3
:0142CA0022D1
:0242CB008F3D25
:1042CD00A2AF9227C2AFE4F5838D82740A122B47F9
:1042DD00E53D43A220122B4953A2DFA22792AF7FC7
:0142ED0001CF
:0142EE0022AD
:1029A700A907E7FFA805EF93C3966008403B74FCAF
:1029B7002FFF80F00F08EF93C3966008402B74FB3E
:1029C7002FFF80E00F08EF93C3966008401B74FA4F
:1029D7002FFF80D00F08EF93D3966008400B74F950
:1029E7002FFF80C01F1F1F1F1FEF54FEF80303F7A1
:1029F700E893FC08E893FD08E893FE08E893FF22B4
:102A070009E993C39D6008402974FB29F980F109FE
:102A1700E993C39E6008401A74FA29F980E209E92C
:102A270093D39F6008400B74F929F980D3191919BA
:102A37001919E9C313C313FF22740093F8ECC39861
:102A47004024701F740193F8EDC3984019701474F3
:0E2A57000293F8EEC398400E7009740393F8D2
:102A6500EFC39840037F00227F0122EDF8E6F008CE
:102A7500A3DFFA22EDF8E0F608A3DFFA22E0A3636C
:102A8500A201F0A363A201DFF475A20022E0A36313
:102A9500A201F0A363A201E0A363A201F0A363A2D4
:102AA50001E463A201F0A363A201DFE175A20022A4
:102AB500E0A363A2016DFE936CFDEE058393FC1507
:102AC5008363A201DFEA75A200227F00E493A3637A
:102AD500A201F00F600CA3E583C2E3F58363A201B5
:102AE50080EA75A20022E0A363A201F0A3E583C2F8
:102AF500E3F58363A201DFEE75A20022E0A363A2E2
:102B050001F0A3E583C2E4D2E3F58363A201DFEC20
:102B150075A20022E583C2E3F583E0A363A201F079
:102B2500A363A201DFEE75A20022E583C2E4D2E32E
:102B3500F583E0A363A201F0A363A201DFEC75A214
:102B45000022F922C002C004C00612FFF0D006D050
:042B550004D0022284
:1040510020536572763A0020547261737353656E12
:10406100644552520A00205265496E6974204341E9
:104071004E0A002043414E283029203E20544F2132
:104081000A0020545520300A0020545520310A00DE
:03001E00E4FF22DA
:1041A200C28DC2AF438901C28C906E5EE0FF700780
:1041B200F58A758CEE8016EFB40508E4F58A758CE5
:1041C200B8800AEFB40A06E4F58A758C70D28CD2F4
:0241D200AF221A
:10409100C28DC2AF438901C28C906E5EE0FF701485
:1040A100302609F58A758CDCC226801E758A6675F4
:1040B1008CFC8016EFB40508E4F58A758CEE800A55
:0F40C100EFB40A06E4F58A758CDCD28CD2AF22FC
:10437100123559124456D225E4F537906F66F0F59F
:0C43810025F53B1241A2C226E4F53922CA
:10410800EF24FCF53D201D127E407F511231E07EE8
:104118006B7F387B01AD3D123481906B3863A2010F
:10412800906EE663A201AF3D122A82853D25E4F533
:0341380036C22369
:01413B002261
:0F43F200D3EF6480948E5006E53B70028F3B2220
:1025B500208D03022652C28C2025030226B5E5256F
:1025C500605474EA2536F582E4346EF583E024051B
:1025D500F53DD3940E4008E4F525D2230226B574C3
:1025E500E62536F582E4346EF5837D27AF3D122A64
:1025F50079E53D2536F536E52730E702D226124145
:10260500A212362FE536C3952550030226B5E4F50B
:1026150025D2230226B5E5386015906E4A7D27FF41
:10262500122A791241A212362FE4F5380226B5E5B1
:102635003B60149068407D27FF122A791241A2124F
:10264500362FE4F53B8069123C961241A21239C837
:102655008F3DEF605B124091E4F539E527547EB577
:102665002703123F67E53AC3946E5018745F253A05
:10267500F582E4346EF583E53D253AF53A7D27AFDD
:102685003D122A70301424E52730E70330021C90F0
:102695006D367D27AF3D122A70AF3D123878EF7049
:1026A5000A201D077E407F581231E0AF3D121E3EC5
:1026B50030201230130D0539E539D394F04004C2AA
:1026C500AF80FEC2202015030227C2E5376031D353
:1026D5009401400415378028906F66E004F0E0D33C
:1026E5009403400D201D077E407F671231E01243A1
:1026F50071201D077E407F741231E0E4F537D22545
:10270500302443E538703F906E4A04F0A37408F016
:10271500A37480F0A37401F0A37406F0906EE1E059
:10272500906E4FF0906EE2E0906E50F0906EE3E0A8
:10273500906E51F0906EE4E0906E52F0E4A3F0A339
:10274500F075380BC224302272906EDFE07035E5EB
:10275500387031906E4A7442F0A37408F0906EE0C0
:10276500E0906E4CF0906EE5E0906E4DF0A3740134
:10277500F0753806201D077E407F831231E0906E8C
:10278500DFE004F0906EDFE06402702FE538702B17
:10279500906E4A7402F0A37408F0906EE0E0906EBB
:1027A5004CF0A3F0A37401F0753806201D077E4098
:1027B5007F8A1231E0906EDFE004F0C21512002628
:0127C50022F1
:10416F00E53A602CE4906C34F0A3E53AF0906E37AA
:10417F00E0906C36F0A37419F0906E5F63A201901B
:10418F006C3863A201AF3A122A82E4F53A7F01221A
:03419F007F00227C
:0B442800302305C2237F01227F002209
:0100210022BC
:06445000E4F53AF5252217
:100006007F01E4906943F0A3F0A3F0FEEF25E0FF43
:040016000EBE08F81A
:01001A0022C3
:0744490020457272210A00F8
:1043A400EF600A7B10E4FD7F0C124254227B107DE7
:0743B400107F0C124254229D
:10355900D29475C353C29475C5C0E5C4B480FB85C4
:10356900C53ED2947DE07F0F124313906E5EE04416
:1035790080FD7F2A1243137D247F291243137D0482
:103589007F28124313E4FD7F2B124313754020E477
:10359900F53FE4FDAF401243130540053FE53FC346
:1035A900940840EEE4F540F53FE4FDAF40124313C3
:1035B9000540053FE53FC3940C40EE7D087F0512A9
:1035C9004313754010E4F53FE4FDAF401243130582
:1035D90040053FE53FC3940C40EE7D3C7F0C124310
:1035E900137D077F0F1243137DFF7F2B1243137542
:1035F9004030E4F53EE4F53FE4FDAF4012431305E6
:1036090040053FE53FC3940E40EE05400540053EA9
:10361900E53EC3940340DE7D047F60124313E4FD5D
:053629007F7012431345
:01362E002279
:1042EF00C29475C503E5C4B480FBAEC58FC5E5C4E4
:1042FF00B480FBAEC5E4F5C5E5C4B480FBAEC5D252
:03430F0094AF0662
:014312002288
:10431300C29475C502E5C4B480FBAEC58FC5E5C4C0
:10432300B480FBAEC58DC5E5C4B480FBAEC5D294E5
:014333002267
:10425400C29475C505E5C4B480FBAEC58FC5E5C47D
:10426400B480FBAEC58BC5E5C4B480FBAEC58DC5BB
:09427400E5C4B480FBAEC5D29490
:01427D00221E
:1033A300C29475C503E5C4B480FBAEC5EF60047E6B
:1033B3007080027E608EC5E5C4B480FBAEC5E4F5C3
:1033C300C5E5C4B480FB85C526E4F5C5E5C4B48072
:1033D300FB85C527E4F5C5E5C4B480FB85C528E4B2
:1033E300F5C5E5C4B480FB85C529E4F5C5E5C4B4DA
:1033F30080FB85C52AE4F5C5E5C4B480FB85C52BF0
:10340300E52B540FFE60741EE4F5C5E5C4B480FBE0
:1034130085C52CEE60651EE4F5C5E5C4B480FB8567
:10342300C52DEE60561EE4F5C5E5C4B480FB85C525
:103433002EEE60471EE4F5C5E5C4B480FB85C52FB9
:10344300EE60381EE4F5C5E5C4B480FB85C530EEF7
:1034530060291EE4F5C5E5C4B480FB85C531EE6083
:103463001A1EE4F5C5E5C4B480FB85C532EE600BD6
:0D347300E4F5C5E5C4B480FB85C533D294F3
:013480002229
:10362F00C29475C502E5C4B480FBAFC575C531E55D
:10363F00C4B480FBAFC5E52B540FFE8527C5E5C489
:10364F00B480FBAFC58528C5E5C4B480FBAFC58585
:10365F0029C5E5C4B480FBAFC5852AC5E5C4B480D0
:10366F00FBAFC5852BC5E5C4B480FBAFC5EE606C61
:10367F001E852CC5E5C4B480FBAFC5EE605E1E850C
:10368F002DC5E5C4B480FBAFC5EE60501E852EC5B9
:10369F00E5C4B480FBAFC5EE60421E852FC5E5C4FF
:1036AF00B480FBAFC5EE60341E8530C5E5C4B48071
:1036BF00FBAFC5EE60261E8531C5E5C4B480FBAFF8
:1036CF00C5EE60181E8532C5E5C4B480FBAFC5EEEC
:1036DF00600A8533C5E5C4B480FBAFC5D2947F02C1
:1036EF00C29475C581E5C4B480FBAFC5D29475375C
:0336FF000AC225D7
:0137020022A4
:103F6700C29475C502E5C4B480FBAFC575C541E50C
:103F7700C4B480FBAFC58527C5E5C4B480FBAFC516
:103F87008528C5E5C4B480FBAFC58529C5E5C4B49C
:103F970080FBAFC5852AC5E5C4B480FBAFC5E4F592
:103FA700C5E5C4B480FBAFC5D2947F02C29475C582
:0A3FB70082E5C4B480FBAFC5D294CC
:013FC10022DD
:103C9600C29475C502E5C4B480FBAFC575C551E5D0
:103CA600C4B480FBAFC574862515F582E43461F58E
:103CB60083E0F5C5E5C4B480FBAFC575C508E5C4AA
:103CC600B480FBAFC574872515F582E43461F583AE
:103CD600E0F5C5E5C4B480FBAFC575C50FE5C4B452
:103CE60080FBAFC50515051574862515F582E434E8
:103CF60061F583E07002F515E4F5C5E5C4B480FB13
:103D0600AFC5D2947F02C29475C584E5C4B480FB66
:043D1600AFC5D294CF
:013D1A002286
:1039C8003092037F00227F2C1242EF8F3EE53E307B
:1039D800E209D225E4F537906F66F0E53E30E55808
:1039E800201D077E447F491231E07F2D1242EF8F60
:1039F8003F201D11E53EFE7C00E4253FFFEC3EFE26
:103A08007D031232C5E4FBAD3F7F2D124254201DC9
:103A18001BE53E30E016E4FF1233A3E527FE7C00E9
:103A2800E4252BFFEC3EFE7D031232C5AB3EE4FDE0
:103A38007F2C1242547F0022E4F53FE53E30E00B34
:103A4800E4FF1233A3E52B2405F53FAB3EE4FD7FED
:063A58002C124254AF3FA6
:013A5E002245
:101AF500C7E0E3F0F3E7EEF7EDFBE920EEE1F0E018
:101B0500E73A20CACF20C8F1E5F2FC28C3F0E0EDA2
:101B1500E8F22DC029207620312E30340A005452A7
:101B2500414E5A004D415842005254530044454CD1
:101B35004159004D4F4445004B5000545500434119
:101B45004E004B5654004154004449520043414E07
:101B55004D4F4E00475254494D450054495453008A
:101B65005453494E5600000A41734F55543A2000CC
:101B750054530A005455204F4B0A005455204469CC
:101B850061670A005455205265710A00205455209A
:101B950054696D654F5554210A004154636F6E6E4B
:101BA5006563740A000A4173494E3A20000A43529C
:101BB50043204552523A20000A4E6B703A20000AE3
:101BC500CFF0E8EDFFF2E020EAEEECE0EDE4E02016
:101BD500D2D320002020D2D320E7E0EDFFF2EE2182
:101BE5000A000ACDE520EFEEEDFFEB20F2E8EF204D
:101BF500EFE0EAE5F2E0210A0000112332465765DD
:101C0500748C9DAFBECADBE9F810013322564775C7
:101C1500649C8DBFAEDACBF9E821300213677644B8
:101C250055ADBC8E9FEBFAC8D931201203776654A7
:101C350045BDAC9E8FFBEAD8C94253617004152798
:101C450036CEDFEDFC8899ABBA5243716014053787
:101C550026DECFFDEC9889BBAA6372405125340678
:101C650017EFFECCDDA9B88A9B7362504135241667
:101C750007FFEEDCCDB9A89A8B8495A7B6C2D3E150
:101C8500F008192B3A4E5F6D7C9485B7A6D2C3F147
:101C9500E018093B2A5E4F7D6CA5B48697E3F2C038
:101CA500D129380A1B6F7E4C5DB5A49687F3E2D027
:101CB500C139281A0B7F6E5C4DC6D7E5F48091A318
:101CC500B24A5B69780C1D2F3ED6C7F5E49081B307
:101CD500A25A4B79681C0D3F2EE7F6C4D5A1B082F8
:101CE500936B7A48592D3C0E1FF7E6D4C5B1A092E7
:101CF500837B6A58493D2C1E0F0089129B24AD3603
:101D0500BF48C15AD36CE57EF78108931AA52CB755
:101D15003EC940DB52ED64FF76028B109926AF3445
:101D2500BD4AC358D16EE77CF5830A9118A72EB535
:101D35003CCB42D950EF66FD74048D169F20A93225
:101D4500BB4CC55ED768E17AF3850C971EA128B315
:101D55003ACD44DF56E960FB72068F149D22AB3005
:101D6500B94EC75CD56AE378F1870E951CA32AB1F5
:101D750038CF46DD54EB62F97008811A932CA53EE5
:101D8500B740C952DB64ED76FF89009B12AD24BFD5
:101D950036C148D35AE56CF77E0A8318912EA73CC5
:101DA500B542CB50D966EF74FD8B029910AF26BDB5
:101DB50034C34AD158E76EF57C0C851E9728A13AA5
:101DC500B344CD56DF60E972FB8D049F16A920BB95
:101DD50032C54CD75EE168F37A0E871C952AA33885
:101DE500B146CF54DD62EB70F98F069D14AB22B975
:101DF50030C74ED55CE36AF1780008040C020A0688
:101E05000E0109050D030B070FFF1B23FF1B29FF00
:101E15001B2EFF1B32FF1B38FF1B3DFF1B40FF1B0B
:101E250043FF1B47FF1B4BFF1B4EFF1B52FF1B595D
:091E3500FF1B60FF1B65FF1B6B26
:1043BB00EF540F901DFE93FEC454F0FEEFC4540F48
:0443CB00932EFF220C
:084433007E1A7FF51231E02230
:030023000237039E
:0B370300C0E0C083C082C0D075D018A9
:10370E0030984EC298755201AF9920074420030994
:10371E00EF6402703CD2038038300C04C20C80225D
:10372E00BF0904D20C802ABF0205530C808022BF31
:10373E000310906613E50CF0630C80530C80C203EB
:10374E00800F7436250CF582E43466F583EFF005B0
:10375E000C30995B300456906185E0FFE50DC39FF8
:10376E004006C204D2118045AF0D050D74362FF5FB
:10377E0082E43467F583E0F510300B1953107F3077
:10378E00012830D008300622631080801D20061AD2
:10379E006310808015300112E50B5210300606A220
:0F37AE00D0929B8005A2D0B3929B851099C299AF
:0937BD00D0D0D082D083D0E032DC
:10162800C20EE4906402F0906838F0D20DC202C293
:1016380005906836F0A37478F0D20AE4906E5EF0F4
:10164800906F7C7461F0A37486F0906F7CE475F001
:101658000112217E85F082F58374C4F0906F7CE4DA
:1016680075F00112217E85F082F583E4F0906F7C9D
:1016780075F00112217E85F082F58374C4F0906FB5
:101688007CE475F00112217E85F082F5837401F007
:10169800906F7CE475F00112217E85F082F58374E9
:1016A800C8F0906F7CE475F00112217E85F082F518
:1016B80083E4F0906F7C75F00112217E85F082F54D
:1016C8008374C8F0906F7CE475F00112217E85F078
:1016D80082F5837401F0906F7CE475F00112217E2D
:1016E80085F082F58374C2F0906F7CE475F0011286
:1016F800217E85F082F583E4F0906F7C75F001120D
:10170800217E85F082F58374C2F0906F7CE475F0D9
:101718000112217E85F082F5837401F0906F7CE4DC
:1017280075F00112217E85F082F583E4F0906F7CDC
:1017380075F00112217E85F082F583E4F0F51590AD
:101748006F74F0906F74E075F003A4240EF582E4D2
:10175800341EF583E493FB740193FA740293F9122F
:1017680020E37003021AF4E4906F76F0A3F0906F10
:1017780075F0906F75E0246BF582E43469F583E0C9
:10178800FF7003021AEB906F74E075F003A4240E47
:10179800F582E4341EF583E493FB740193FA740232
:1017A80093F9906F76E0F5827583001220FCFEEFC6
:1017B800B5060F906F777401F0906F76E004F00231
:1017C8001AE2906F77E07003021AE2EE6003021AE1
:1017D800D9906F74E0B40F004003021AEB9017EC35
:1017E800F828287302181902186602197D0219824E
:1017F8000219B1021A18021AEB0219E7021AEB02CF
:101808001A49021A9D021ACD021AD1021AEB021ABB
:10181800D5906F75E0246BF9E43469FA7B01C00355
:101828001B8B40754100754200E4F543D003122B31
:1018380059906F78122281906F78E0F8A3E0F9A3AD
:10184800E0FAA3E0FB7F007E8C7D0A7C001221D0A9
:1018580012226290683AEEF0A3EFF0021AEB906F52
:101868007C7461F0A37486F0906F75E0246BF58248
:10187800E43469F583E024D0F515C394014007E505
:1018880015D394084003E4F515E5156028906F7C9E
:10189800E475F00112217E85F082F58374C4F01599
:1018A80015906F7CE475F00112217E85F082F58336
:1018B800E515F080D4906F75E0246CF582E4346906
:1018C800F583E024D0F515C394014007E515D394BA
:1018D800084003E4F515E5156028906F7CE475F081
:1018E8000112217E85F082F58374C8F01515906F7A
:1018F8007CE475F00112217E85F082F583E515F010
:1019080080D4906F75E0246DF582E43469F583E046
:1019180024D0F515C394014007E515D39408400376
:10192800E4F515E5156028906F7CE475F001122147
:101938007E85F082F58374C2F01515906F7CE4758E
:10194800F00112217E85F082F583E515F080D490B0
:101958006F7CE475F00112217E85F082F583E4F056
:10196800906F7C75F00112217E85F082F583E4F09A
:10197800F515021AEBD20F021AEB906F75E0246B83
:10198800F9E43469FA7B01C0031B8B40754100758B
:101998004200E4F543D003122B59906F781222814C
:1019A800906F7BE0F509021AEB906F75E0FF246BEE
:1019B800F582E43469F583E0B43702D20B746C2FF6
:1019C800F582E43469F583E0FFB44E04C201800275
:1019D800D201EF64456003021AEBD206021AEB90BB
:1019E8006F75E0246BF9E43469FA7B01C0031B8B43
:1019F80040754100754200E4F543D003122B59901D
:101A08006F78122281906F7BE0906E5EF0021AEB85
:101A1800906F75E0246BF9E43469FA7B01C0031B0D
:101A28008B40754100754200E4F543D003122B59F1
:101A3800906F78122281906F7BE0906402F0021A16
:101A4800EB906F75E0246BF9E43469FA7B01C0030D
:101A58001B8B40754100754200E4F543D003122BFF
:101A680059906F78122281E4FFFEFDFC906F78E0B8
:101A7800F8A3E0F9A3E0FAA3E0FBD3122270400F29
:101A8800906F7AE0FFA3E0906836CFF0A3EFF0D232
:101A98000EC20D804E906F75E0246BF9E43469FA3C
:101AA8007B01C0031B8B40754100754200E4F54380
:101AB800D003122B59906F78122281906F7BE0909F
:101AC8006838F0801ED202801AD2058016C20A80B9
:101AD80012E4906F77F0906F76F0906F75E004F0F5
:0C1AE80002177A906F74E004F002174BB4
:011AF40022CF
:1030ED00C222C210C209C208906182740AF0E49033
:1030FD006839F0906837E024F9FE906836E034FFC7
:10310D00906300F0A3CEF0E4906184F0C21290665B
:10311D00157405F0C224E4F508906941E06455701A
:10312D0004A3E06481603BE4FF7F409061B6E4F06E
:10313D00A3DFFCE4FF7F20906616E4F0A3DFFCE440
:10314D00FF74032FF582E43466F583E4F0740B2FDE
:10315D00F582E43466F583E4F00FBF08E4E4F50E80
:10316D00F50FE4F514F5139062FFF09062FEF0C2D6
:10317D0004C211C207C203C20CF50D906185F0F5B2
:10318D0009F50CF552C200C20BC20F90683A74FFDC
:10319D00F0A374F4F0750BFF121628E4F59BC2AD85
:1031AD00F5C9D2CDD2CCC2C9C2CAF5CDF5CC906885
:1031BD003AE0F5CBA3E0F5CA85CBCD85CACCD29E3E
:1031CD00D29CD2CAC2ACC298C29975B81075B7104C
:0231DD00D2AC72
:0131DF0022CD
:1043CF00E5126FFF901CFE936511F512EF901BFE27
:0343DF0093F51142
:0143E20022B8
:0237C6008F432F
:1037C800E4FC754461754500F512F511FDEDC395EE
:1037D8004350170545E545AE447002054414F5828B
:1037E8008E83E0FF1243CF0D80E30545E545AE44E7
:1037F8007002054414F5828E83E512F085458285B2
:103808004483E511F0054305437E677F36754461BF
:103818007545008F828E837402F00FBF00010E0C75
:10382800E4FDEDC395435038854582854483E0F92E
:1038380064026008E964036003B9090D8F828E830E
:103848007409F00FBF00010E0C8F828E83E9F00F10
:10385800BF00010E0C0545E545700205440D80C208
:0F3868008F828E837403F00FBF00010E0CAF042C
:01387700222E
:03445600C2072278
:10400E008F4220043D300D3AAF421237C690618583
:10401E00EFF0201D127E1B7F6C1231E07E617F005F
:10402E00E4FBAD42123481300F057F011243A4E54B
:10403E00096003F54F22E4F50DD204C2992099FDD3
:03404E00D29922E2
:021E3E008F3ED5
:101E4000906402E070030220E2E52724BE700302E2
:101E5000208B24FA700302200F240460030220E286
:101E6000E52830E703021EFAE52A6068E529C394F5
:101E70000240030220E2E5297007E52A14F53F80BD
:101E800006E52A241FF53FE53F75F004A42402F57A
:101E900082746335F0F5837D2C7F04122A70E53F50
:101EA00075F004A424FEF582746135F0F5837D306D
:101EB0007F04122A7074F62529F582E43461F583D3
:101EC0007481F074B6253FF582E43461F5837401C2
:101ED000F0D2082274032529F582E43466F5837470
:101EE00080F0E52975F004A42416F582746635F0B7
:101EF000F5837D2C7F04122A7022E52B6408600391
:101F00000220E2E529C3940440030220E2201D07D9
:101F10007E1B7F751231E0753E01E52A5407FFE50F
:101F20003EA807088002C333D8FCF53E7408250F8D
:101F3000F50FB50E067408250EF50EE52A547FFF41
:101F4000E529C43354E02FFE7400250FF582E434F4
:101F500060F583EEF0E52AC394805022EF1313134B
:101F6000541FFFE52925E025E02F2416F582E434EF
:101F700066F583E0FFE53EF4FEEF5EF0802EE52A95
:101F8000547FFF131313541FFFE52925E025E02F8D
:101F90002416F582E43466F583E0453EF0740025AE
:101FA0000FF582E43460F583E04480F07401250F7E
:101FB000F582E43460F5837D2C7F04122A70E531CC
:101FC000FEE530FF7C007D0A122129EF7405250F04
:101FD000F582E43460F583EFF07406250FF582E4B2
:101FE0003460F583E532F07407250FF582E4346040
:101FF000F583E533F0301D030220E27400250FF570
:1020000082E43460AF82FEE4FB7D0812348122E575
:102010002A54E0644070030220E2E529701DE52A9D
:102020001313543FFF7401A807088002C333D8FC80
:1020300042139062FEE04513F08024E529640160BC
:10204000030220E2E52A1313543FFF7401A8070896
:102050008002C333D8FC42149062FFE04514F0E5DF
:102060002975F020A4FFE52A547F7C002FFFEC3572
:10207000F0FEEF25E0FFEE33FE74032FF58274646B
:102080003EF5837D2CAF2B122A7022E52AB4011372
:10209000201D077E1B7F791231E0E52D04906F67CC
:1020A000F0C222E52AB40216240BF582E43466F568
:1020B00083E52DF0201D077E1B7F801231E0E52A8D
:1020C000B4031F240BF582E43466F583E52DF0207C
:1020D0001D077E1B7F891231E0302206906EDF746F
:0220E00002F00C
:0120E20022DB
:10002600906402E07003020A19301361050A9066B3
:1000360015E0600214F0906839E0600214F09068F0
:1000460038E06008906182E0600214F0C213300E5E
:1000560021906836E0FEA3E0FFD3906301E09F9015
:100066006300E09E500CA3E004F07006906300E08D
:1000760004F0302218906183E004F0E0D3940A4043
:100086000C201D077E1B7F911231E0C222E54FB482
:10009600010EE4F54FF50DD204C2992099FDD299CF
:1000A60030040DE50AD394064009C204D211800338
:1000B600E4F50A200E03020191906837E024FBFF65
:1000C600906836E034FFFEC3906301E09F906300C2
:1000D600E09E4012906184E0700CC20DFF1243A4B2
:1000E6009061847401F0906837E024FDFF906836D3
:1000F600E034FFFEC3906301E09F906300E09E4002
:1001060012906184E0B4010B7F011243A4906184D4
:100116007402F0906837E024FEFF906836E034FF02
:10012600FEC3906301E09F906300E09E405D200463
:100136005A9067367441F0A37454F0A37424F0A364
:100146007443F0A3744FF0A314F0A3F0A37445F026
:10015600A37443F0A37454F0A3740DF0A3740AF0CF
:10016600906185740CF0E4F50DD204C2992099FDD6
:10017600D299E4906300F0A3F0906184F0301D03FF
:10018600020A197E1B7F9F1231E02230110AC2112A
:10019600300F05E4FF1243A4300403020678E54F4E
:1001A6006003020678200D03020678906182E06003
:1001B60003020678906838E06007E4906182F08078
:1001C60006906182740AF0301229C212E49061002E
:1001D600F0A37408F0906402E0906102F090661457
:1001E600E0906103F0A374FEF0A3748FF07F061213
:1001F600400E22906F67E0FF6025E4906100F0A357
:100206007408F0906402E0906102F0A37483F0A396
:10021600EFF0E4A3F0906F67F07F0612400E22E540
:100226000F650E7003020326906839E0600302042E
:1002360012E50E2408F53EE4906100F0A37408F080
:10024600906402E0906102F0A374F0F0A37406F0EB
:10025600A37491F07406253EF582E43460F583E0DC
:10026600906106F07407253EF582E43460F583E07C
:10027600906107F07401253EF582E43460F583E071
:10028600906108F07402253EF582E43460F583E05F
:10029600906109F07403253EF582E43460F583E04D
:1002A60090610AF07404253EF582E43460F583E03B
:1002B60090610BF07400253EF582E43460F583E02E
:1002C600FF547FFEC39440500BEFC454F00490617A
:1002D6000CF080167400253EF582E43460F583E068
:1002E600FFC454F0240590610CF07400253EF5829D
:1002F600E43460F583E0FFEEC4540F90610DF0EF37
:100306005480FF7405253EF582E43460F583E02FC2
:1003160090610EF09068397414F07F0F12400E222F
:10032600300973906603E0D39400406AE49061005C
:10033600F0A37408F0906402E0906102F0A37441A7
:10034600F0A37420F0754061754105E4F53E74161E
:10035600253EF582E43466F583E0F53F300A06FF74
:100366001243BB8F3F854182854083E53FF0F4FF12
:10037600E5822408F582E43583F583EFF00541E54F
:100386004170020540053EE53EC3940840C07F1516
:1003960012400EC20922301073906605E0D3940015
:1003A600406AE4906100F0A37408F0906402E09063
:1003B6006102F0A37445F0A37420F07540617541A5
:1003C60005753E087416253EF582E43466F583E02D
:1003D600F53F300A06FF1243BB8F3F8541828540B9
:1003E60083E53FF0F4FFE5822408F582E43583F5E2
:1003F60083EFF00541E54170020540053EE53EC349
:10040600941040C07F1512400EC21022200803022D
:1004160005159061F7E0FF9061F6E04F5401D39423
:10042600005003020515E4F53E74B6253EF582E458
:100436003461F583E0700302050774B6253EF58244
:10044600E43461F583E4F0906100F0A37408F09061
:100456006402E0906102F0A374F0F0A37403F0A3C9
:100466007491F0E53EC4540F2408A3F0E53E540F02
:10047600A3F0E53E25E025E0F53E24FEF582E434D2
:1004860061F583E0906108F074FF253EF582E4345F
:1004960061F583E0906109F07400253EF582E4344D
:1004A60062F583E090610AF07401253EF582E4343A
:1004B60062F583E090610BF0E4A3F07402253EF54B
:1004C60082E43463F583E090610DF07403253EF514
:1004D60082E43463F583E090610EF07404253EF502
:1004E60082E43463F583E090610FF07405253EF5F0
:1004F60082E43463F583E0906110F07F1112400EC0
:1005060022053EE53EC39440500302042FC20890E4
:100516006615E0704130053E7478F0E4906100F0B5
:10052600A37408F0906402E0906102F0A374F0F006
:10053600E4A3F0A37490F0A37408F0E4A3F0A3F08E
:10054600A3F0A3F0A3F0A3F0A3F0A3F0A3F0A3F00D
:100556007F1112400E22E508C394045070E5082569
:10056600E0FF7403A807088002C333D8FCF53E55A4
:1005760013653E7053E53EF45213E4906100F0A318
:100586007408F0906402E0906102F0A374F0F0A3A6
:100596007402F0A37491F0E5082420A3F0E5083373
:1005A600333354F875F002A42403F582E5F034647D
:1005B600F58363A20190610763A2017F10122A826C
:1005C6007F1712400E0508220508020653E508C3E8
:1005D60094085076E50824FC25E0FF7403A8070874
:1005E6008002C333D8FCF53E5514653E7058E53E8F
:1005F600F45214E4906100F0A37408F0906402E0F1
:10060600906102F0A374F0F0A37402F0A37491F069
:10061600E50854032440A3F0E50833333354F87552
:10062600F002A42403F582E5F03464F58363A201A5
:1006360090610763A2017F10122A827F1712400E73
:1006460005085308072205088003E4F50890683872
:10065600E0701F906100F0A37408F0906402E090CF
:100666006102F0A37490F0E4A3F0A3F07F061240B9
:100676000E22906613E0FF7003020A19F53FE4F0BC
:10068600201D1F7E1B7FAA1231E0E53F54802436D1
:10069600F582E43466AF82FEE53F547FFDE4FB124B
:1006A6003481E53F7003020A19E53F5480FF243682
:1006B600F582E43466AD82F5408D41E4F512F5111C
:1006C6008F3EE53EC3953F50180541E541AE40706B
:1006D60002054014F5828E83E0FF1243CF053E806B
:1006E600E1E51145126026301D03020A197E1B7FC3
:1006F600B21231E0E53F54802436F582E43466AF29
:1007060082FEE53F547FFDE4FB12348122E49063D0
:1007160000F0A3F0D20D906184F0E53F54802436BA
:10072600F582E43466AF82F5408F4174022541F5C7
:1007360041E43540F540854182F583E0FF9064024F
:10074600E0FEEF6E6026301D03020A197E1B7FBD98
:100756001231E0E53F54802436F582E43466AF82F8
:10076600FEE53F547FFDE4FB123481220541E5415D
:1007760070020540F582854083E0FFB43006E490C0
:100786006182F022EF64017003020A19EFB41805C2
:10079600D209D21022EFB4190B9062FEE0F513A332
:1007A600E0F51422854182854083E0FF54F064F031
:1007B60060030208A1906614EFF00541E54170025E
:1007C6000540F582854083E0FF648070330541E58E
:1007D6004170020540F582854083E0644060030273
:1007E6000A19D2120541E54170020540F58285409D
:1007F60083E064086003020A19D205906615F022A8
:10080600EFB401270541E54170020540F5828540B8
:1008160083E0644F6003020A19906839E0700302AE
:100826000A197408250EF50EE4F0228541828540EA
:1008360083E06003020A190541E54170020540F5AF
:1008460082854083E064426003020A190541E5415E
:1008560070020540F582854083E0906EE1F0054127
:10086600E54170020540F582854083E0906EE2F036
:100876000541E54170020540F582854083E0906EB2
:10088600E3F00541E54170020540F582854083E0CD
:10089600906EE4F0D224C205D212228541828540B0
:1008A60083E0FF64116008EF641260030209F7E554
:1008B6003F547F640E60030209F7201D077E1B7FED
:1008C600C41231E030220E301D03020A197E1B7F4E
:1008D600D91231E022854182854083E0540314F524
:1008E6003F0541E54170020540F582854083E0F50C
:1008F6003E30E709E4906EE0F0906EE5F0E53E30BC
:10090600E60BE4906EE0F0906EE57410F0E53E3094
:10091600E50B906EE07401F0E4906EE5F0E53E3094
:10092600E40C906EE07401F0906EE57410F0E53E14
:1009360030E30B906EE07402F0E4906EE5F0E53E75
:1009460030E20C906EE07402F0906EE57410F0E503
:100956003E30E10B906EE07403F0E4906EE5F0E556
:100966003E30E00C906EE07403F0906EE57410F08B
:1009760074022541F541E43540F540854182F58311
:10098600E0F53E30E700E53E30E607906EE5E02410
:1009960002F0E53E30E507906EE5E02404F0E53E22
:1009A60030E407906EE5E02406F0E53E30E307907C
:1009B6006EE5E02408F0E53E30E207906EE5E024BF
:1009C6000AF0E53E30E107906EE5E0240CF0E53EE6
:1009D60030E007906EE5E0240EF0906EE5E0253FEE
:1009E600F0D222E4906183F0906EDFF0906F67F0B2
:1009F60022201D1F7E1B7FE71231E0E53F54802435
:100A060036F582E43466AF82FEE53F547FFDE4FBB3
:030A160012348116
:010A190022BA
:103B9000020A1AE493A3F8E493A34003F68001F227
:103BA00008DFF48029E493A3F85407240CC8C33336
:103BB000C4540F4420C8834004F456800146F6DF05
:103BC000E4800B010204081020408090443BE47E16
:103BD000019360BCA3FF543F30E509541FFEE493FA
:103BE000A360010ECF54C025E060A840B8E493A3C1
:103BF000FAE493A3F8E493A3C8C582C8CAC583CAEC
:103C0000F0A3C8C582C8CAC583CADFE9DEE780BEA3
:01444100007A
:1020E300BB010689828A83E0225002E722BBFE02FB
:0920F300E32289828A83E493222E
:1020FC00BB010CE58229F582E5833AF583E0225099
:10210C0006E92582F8E622BBFE06E92582F8E222E2
:0D211C00E58229F582E5833AF583E49322FC
:10212900BC000BBE0029EF8DF084FFADF022E4CC9A
:10213900F875F008EF2FFFEE33FEEC33FCEE9DEC63
:10214900984005FCEE9DFE0FD5F0E9E4CEFD22EDA9
:10215900F8F5F0EE8420D21CFEADF075F008EF2FF3
:10216900FFED33FD4007985006D5F0F222C398FDE4
:052179000FD5F0EA2281
:10217E00A3F8E0C5F025F0F0E58215827002158314
:06218E00E0C838F0E82271
:1021940075F008758200EF2FFFEE33FECD33CDCC02
:1021A40033CCC58233C5829BED9AEC99E582984085
:1021B4000CF582EE9BFEED9AFDEC99FC0FD5F0D662
:1021C400E4CEFBE4CDFAE4CCF9A88222B800C1B98C
:1021D4000059BA002DEC8BF084CFCECDFCE5F0CBCA
:1021E400F97818EF2FFFEE33FEED33FDEC33FCEB03
:1021F40033FB10D703994004EB99FB0FD8E5E4F9BE
:10220400FA227818EF2FFFEE33FEED33FDEC33FCAA
:10221400C933C910D7059BE99A4007EC9BFCE99A9E
:10222400F90FD8E0E4C9FAE4CCFB2275F010EF2FE3
:10223400FFEE33FEED33FDCC33CCC833C810D707E3
:102244009BEC9AE899400AED9BFDEC9AFCE899F81E
:0E2254000FD5F0DAE4CDFBE4CCFAE4C8F922B1
:0E226200C3E49FFFE49EFEE49DFDE49CFC228D
:10227000EB9FF5F0EA9E42F0E99D42F0E89C45F0C4
:01228000223B
:0C228100ECF0A3EDF0A3EEF0A3EFF022D0
:10228D00A8828583F0D083D0821222A41222A412B8
:10229D0022A41222A4E473E493A3C583C5F0C583DD
:1022AD00C8C582C8F0A3C583C5F0C583C8C582C89B
:0122BD0022FE
:102B59008B3D8A3E893FE4F549F548F547F546F549
:102B690044F545E541454245406012EBC0E0EAC005
:102B7900E0E9C0E0AB40AA41A94212230DAB3D05F3
:102B89003FE53FAA3E7002053E14F91220E3F54ADB
:102B9900C394094007E54AD3940D40E1E54A64200E
:102BA90060DBE54AB42D054345038016E54AB42B9D
:102BB90005434501800C74FF253FF53F74FF353E01
:102BC900F53EE54360046410703FAB3DAA3EA93F62
:102BD9001220E364306009E543702E75430A8029A9
:102BE9009000011220FCFF64786004EFB45813438D
:102BF90045017543107402253FF53FE4353EF53E26
:102C09008007E5437003754308AB3D053FE53FAADF
:102C19003E7002053E14F91220E3F54AC39461405F
:102C29000AE54AD3947A5003534ADF74D0254AF50A
:102C39004AC3940A400CE54A9411406D74F9254A37
:102C4900F54AE54AD39543506043450185494E8588
:102C5900484D85474C85464BAF437E00E4FCFDABB0
:102C690049AA48A947A8461222BEC8ECC8C9EDC955
:102C7900CAEECACBEFCBE4FCFDFEEB254AF549EEE3
:102C89003AF548ED39F547EC38F546AF49AE48AD68
:102C990047FCAB4EAA4DA94CA84BD3122270500346
:102CA900022C12434504022C12E54520E003E4807E
:102CB9002DE54145424540601EAB3DE53F24FFF906
:102CC900E53E34FFFAEBC0E0EAC0E0E9C0E0AB4022
:102CD900AA41A94212230DE54530E20774FFFFFE20
:102CE900FDFC22E545AF49AE48AD47AC4630E103AE
:042CF900022262222F
:1022BE00E88FF0A4CC8BF0A42CFCE98EF0A42CFCBF
:1022CE008AF0EDA42CFCEA8EF0A4CDA8F08BF0A43D
:1022DE002DCC3825F0FDE98FF0A42CCD35F0FCEB9C
:1022EE008EF0A4FEA9F0EB8FF0A4CFC5F02ECD3961
:0F22FE00FEE43CFCEAA42DCE35F0FDE43CFC22CE
:10230D00BB011A89828A83D0F0D0E0F8D0E0F9D0F1
:10231D00E0FAD0E0FBE8C0E0C0F00223655016E91A
:10232D00F8D083D082D0E0F9D0E0FAD0E0FBC082C3
:10233D00C08302235CBBFE16E9F8D083D082D0E0C7
:0F234D00F9D0E0FAD0E0FBC082C08302236E22F9
:09235C00EBF608EAF608E9F622A6
:09236500EBF0A3EAF0A3E9F02279
:09236E00EBF208EAF208E9F222A0
:00000001FF
